:100000000C9430050C9491050C9442080C949105C5
:100010000C9491050C9491050C9491050C94910508
:100020000C9491050C9491050C9452120C9491052A
:100030000C9471210C9491050C9491050C949105EC
:100040000C9491050C9491050C9491050C949105D8
:100050000C9491050C94E1210C9491050C9491055C
:100060000C9491050C9491050C9491050C949105B8
:100070000C9491050C9491050C9491050C949105A8
:100080000C9491050C9491050C9491050C94910598
:100090000C9491050C9491050C9491050C94910588
:1000A0000C9491050C9491050C94910578097A09AA
:1000B0008609860986098609860986097C097E09DA
:1000C0008009860986097A0988098609860942090C
:1000D0007809860986097E098609860986098609BE
:1000E00086098609800978096409860968098609EC
:1000F0008609860944097C098609860972098609E8
:1001000086098609460984098609660986097A09E5
:100110008609860976096A0986096C097E098609B5
:100120008609860974096E09860986098609860981
:10013000860986098609700986094809860986099B
:100140007C09860986098409860986098609860943
:10015000860986098609860986094A098609860963
:10016000860972098609860986098609860986092B
:1001700086098609860986094C0986094E095009AF
:1001800086098609860952095409560986095809BB
:100190005A0986098609860982095C098609600967
:1001A0005E09620986098609860986098409AC09FF
:1001B000BA09C609C6099E09C609C609C609C609FB
:1001C000C609C609C609C609C609C609C609C609B7
:1001D000C609A009C609A209C609C609C609C609F1
:1001E000BE09C609D109BC09C609C609C609C6099E
:1001F000C609C609C609C609C609C609C609C60987
:10020000C6099609B209A409B609C609A609C6090C
:10021000AA09C609B409A809B809AE09B009C609EE
:10022000C609C609C609C609C609C60998099A09B0
:100230009C09C009C209C609C609C609C409AC0B94
:10024000070CEF0B190C2A0C340C390C3D0C440C28
:1002500048136A135D146A135D14AF13D2135D144F
:1002600027143A146D176D1797179717F2171D1A61
:100270001D1A1D1A26181D1A11191119D7191D1A20
:10028000EC190A1A807B01484746293A687F0277B1
:10029000762B353B6978796439141E3C6A7A1D16D1
:1002A000041A1F3D6B061B070821203E6C2C190900
:1002B0001715223F6D11050B0A1C23406E7E100D91
:1002C000182425416F360E0C122726427037380F3E
:1002D00033132D43717534322F2E44727C7D2830B8
:1002E00031744573515065524C4D2A4900594F5C49
:1002F0005F4E4A4B62635A5D5E60535467585B665B
:10030000576155564842403E3C3A3B456843413F61
:100310003D2B357E697A790078141E7C6A7B1D1628
:10032000041A1F7F6B061B070821204D6C2C19092E
:100330001715224A6D11050B0A1C234C6E49100D2E
:10034000182425516F360E0C1227264F7037380FA0
:1003500033132D52717534502F2E4E72397D283043
:1003600065314B735464586776012A773259745C4F
:100370005F66024662635A5D5E60295344575B566E
:100380005561470380291E1F20212223242526276B
:100390002D2E2A2B141A0815171C180C12132F3087
:1003A0002878041607090A0B0D0E0F3334357931FE
:1003B0001D1B06190511103637387D557A2C393A30
:1003C0003B3C3D3E3F4041424353475F6061565C8A
:1003D0005D5E57595A5B62634648324445677B7F8E
:1003E000650301025250514F68696A6B6C6D6E6F04
:1003F0007071725800494C754A4D734B4E767C773C
:100400007E7466547225303258200072253032587E
:10041000200077253032582000214353335F463087
:100420005F25303258210A00214353335F46305F45
:1004300025303258210A00214353335F253032588A
:10044000210A00214353335F25303258210A00210D
:100450004353325F45305F4630210A002143533217
:100460005F4630210A00214353325F4530210A00A4
:10047000214353325F494E4954210A0021435332EC
:100480005F4F56455252554E210A00214353315F6A
:100490003F210A006B62643A20556E6B6E6F776E77
:1004A0000A006B62643A205465726D696E616C0A71
:1004B000006B62643A2041540A006B62643A20582F
:1004C000540A004D6F7573653A206E6F7420737512
:1004D00070706F727465640A0049443A20253034A4
:1004E000580A006572723A20253032580A00696E47
:1004F00069740A006572723A20253032580A000A7F
:100500004B6579626F6172642073746172742E0A34
:10051000000A55534220636F6E66696775726564A1
:100520002E0A000A0A544D4B3A35613735393835B1
:10053000302F4C5546410A0A003403490042004D11
:100540000020005000430020006B0065007900622D
:10055000006F00610072006400200063006F006E95
:100560000076006500720074006500720000000EE5
:100570000374002E006D002E006B002E000000049E
:1005800003090409027400040100A03209040000F8
:1005900001030101000921110100012240000705AA
:1005A000810308000A090401000103000000092179
:1005B000110100012236000705820308000A090420
:1005C00002000203000000092111010001222200A3
:1005D0000705830320000107050303200001090428
:1005E000030001030000000921110100012239006C
:1005F000070584032000011201100100000008ED2E
:10060000FEEE1B01000102000105010906A1010522
:100610000719E029E71500250195087501810205F4
:100620000819012905950575019102950175039138
:10063000010507190029F71500250195F8750181B5
:1006400002C00631FF0974A1010975150026FF00DB
:100650009520750881020976150026FF0095207502
:10066000089102C005010980A1018502160100263A
:1006700037001A81002AB700751095018100C00566
:100680000C0901A1018503160100269C021A010034
:100690002A9C02751095018100C005010906A1017F
:1006A000050719E029E71500250195087501810264
:1006B0009501750881010508190129059505750140
:1006C00091029501750391010507190029FF150095
:1006D00026FF00950675088100C0636F6E73756D07
:1006E00065723A20253034580A0073797374656D49
:1006F0003A20253034580A000A00253032582000AC
:100700006B6579626F6172643A20004C45443A200F
:10071000253032580A00253032583A2025303862C8
:1007200025730A00722F6320303132333435363767
:100730000A0064656C5F6B65795F6269743A206377
:10074000616E27742064656C3A20253032580A00A7
:100750006164645F6B65795F6269743A2063616E9E
:100760002774206164643A20253032580A003F0023
:10077000433E20004C25640A000A092D20436F6E79
:10078000736F6C65202D0A4553432F713A097175BB
:1007900069740A000A092D204D61676963202D0ADA
:1007A000643A0964656275670A783A096465627536
:1007B00067206D61747269780A6B3A0964656275C5
:1007C00067206B6579626F6172640A6D3A096465CE
:1007D000627567206D6F7573650A763A0976657282
:1007E00073696F6E0A733A097374617475730A637F
:1007F0003A09636F6E736F6C65206D6F64650A30C4
:100800002D343A096C61796572302D3428463130C7
:100810002D4634290A506175733A09626F6F746C02
:100820006F616465720A6E3A094E4B524F0A003F7F
:10083000004E4B524F3A206F66660A004E4B524FA5
:100840003A206F6E0A0074696D65725F726561644B
:10085000333228293A202530346C580A006B6579E8
:10086000626F6172645F6E6B726F3A2025580A0086
:100870006B6579626F6172645F69646C653A2025AB
:10088000580A006B6579626F6172645F70726F7491
:100890006F636F6C3A2025580A00686F73745F6B42
:1008A0006579626F6172645F6C65647328293A20B0
:1008B00025580A000A092D20537461747573202D80
:1008C0000A004743433A20352E342E3020415652F9
:1008D0002D4C4942433A20322E302E302041565280
:1008E0005F415243483A20617672350A004F5054B6
:1008F000494F4E533A204C55464120455854524199
:100900004B455920434F4E534F4C4520434F4D4D7F
:10091000414E44204E4B524F204B45594D41505F64
:1009200053454354494F4E20424F4F544C4F41443E
:1009300045525F53495A450A004255494C443A20B2
:100940003561373539383530202830393A30333A47
:100950003232204465632020352032303139290A73
:10096000005649443A2030784645454428742E6D57
:100970002E6B2E29205049443A203078316265652B
:100980002849424D205043206B6579626F61726443
:1009900020636F6E76657274657229205645523AEF
:1009A000203078303030310A00444553433A2063D8
:1009B0006F6E766572742049424D205043206B65FE
:1009C00079626F61726420746F205553420A000A85
:1009D000092D2056657273696F6E202D0A000A6D0D
:1009E0006F7573653A206F66660A000A6D6F7573DE
:1009F000653A206F6E0A000A6B6579626F617264F6
:100A00003A206F66660A000A6B6579626F617264EC
:100A10003A206F6E0A000A6D61747269783A206F2D
:100A200066660A000A6D61747269783A206F6E0A10
:100A3000000A64656275673A206F6E0A000A646591
:100A40006275673A206F66660A000A0A626F6F7401
:100A50006C6F616465722E2E2E2000433E200000D4
:100A600011241FBECFEFDAE0DEBFCDBF04B603FE18
:100A700041C08091980390919903A0919A03B091FD
:100A80009B038730904BA740B04BA1F51092980381
:100A90001092990310929A0310929B0314BE0FB602
:100AA000F894A8958091600088618093600010920E
:100AB00060000FBE1092010810920008E3E0F0E021
:100AC00089E080935700E491E695E370E150E330CC
:100AD00040F4F0E0EE0FFF1FE25DFE4F8081918158
:100AE00002C080E090E1E0E0F0E8E81BF90BF69549
:100AF000E795099511E0A0E0B1E0EAECF7E402C067
:100B000005900D92A433B107D9F723E0A4E3B1E037
:100B100001C01D92A839B207E1F70E94100F0C9492
:100B2000E3230C940000FF93EF93E0913401F091E4
:100B30003501309709F00995EF91FF910895FC0177
:100B40008591803011F0EFDFFBCF0895FF27E0E2C1
:100B500030E247FF0CC0419597FF09C0EDE2609578
:100B6000709580959095611D711D811D911D27FFC8
:100B700002C0219530E350E2AA27660F771F881F35
:100B8000991FAA1FA41710F0A41B63955A95A9F7E3
:100B9000AA3008F0A95FA05DAF93F39561157105C8
:100BA0008105910541F7ED3211F4EF93F395F217BA
:100BB00018F43F93F395FBCF8F91B5DFFA95E1F7EA
:100BC0000895E991F9918591803021F0853219F0ED
:100BD000AADFF9CF089520E0E89455915532C1F38A
:100BE000503311F4689455915A3348F4505390F3AC
:100BF000220F022E220F220F200D250FF4CF0EF40C
:100C0000219589919991533619F3533729F1533529
:100C100059F1BC0188279927E8945C3621F4899121
:100C2000999168945591543639F446EF7EF077FFE8
:100C30000DC08FEF9FEF0AC055374AE039F05835A5
:100C400040E121F0523642E009F00895FF93EF931E
:100C50007DDFEF91FF91B7CFFF93EF93FC0181917F
:100C60008030B9F360DFFBCFFF93EF9368DFF1CF04
:100C7000DF93CF93CDB7DEB72596A3DFCF91DF917A
:100C80000895282F80915201823071F08330B1F0A5
:100C9000813001F5E62FF0E038E0739FE00DF11DA3
:100CA0001124EC57FC4F13C0E62FF0E088E0789F4A
:100CB000E00DF11D1124EC5FFC4F09C0E62FF0E0C0
:100CC00038E0739FE00DF11D1124EC57FD4FE491C6
:100CD000E03819F480E090E008959E2F9077892FF6
:100CE00090E034E0959587953A95E1F738E0239FB9
:100CF000800D911D112444E0880F991F4A95E1F75A
:100D0000EF709C012E0F311DF901EE0FFF1FE05017
:100D1000F8498591949108955998519A0895519858
:100D2000599A08955898509A08955098589A089545
:100D30005198599A85E08A95F1F7000089B1869516
:100D4000817008955098589A85E08A95F1F70000CF
:100D500089B181700895CF93DF93EC010E949806CA
:100D6000882341F0209731F085E08A95F1F7000063
:100D70002197F4CFCE01DF91CF910895CF93DF93E8
:100D8000C2E3D0E00E949806811108C0209731F09C
:100D900085E08A95F1F700002197F4CFCE01DF912D
:100DA000CF9108952091030130E0B9016F5F7F4F2B
:100DB00090910501492F50E046235723609104018B
:100DC00070E04617570791F04091010150910201E0
:100DD000FA01E20FF31F8083809103018F5F9091EE
:100DE000050189238093030181E0089580E008953F
:100DF0000E948C060E9495060E948F060E9495060E
:100E0000E9E6F0E0808188608083E99A0895CF93D5
:100E1000DF939AE19150209103018091040199237D
:100E200049F0281307C0EFE9FFE03197F1F700C060
:100E30000000F0CF281701F1E0910101F0910201CB
:100E4000E80FF11D20818F5F909105018923809328
:100E50000401C22FD0E08091850380FF0FC01F9254
:100E60002F938BE094E09F938F930E9438060F900E
:100E70000F900F900F9002C0CFEFDFEFCE01DF9108
:100E8000CF910895EF92FF920F931F93CF93DF932B
:100E900010923A0190913B01913009F4BCC0C82FE7
:100EA0008091850380FF0CC01F92CF9382E194E074
:100EB0009F938F930E9438060F900F900F900F9082
:100EC000E9980E948C060E9495068FE891E00197B0
:100ED000F1F700C000000E9492060E948F0680E198
:100EE00097E20E94AB06892B11F481E07AC000E002
:100EF00010E0FF24F394D0E0EE24E39490E59A957B
:100F0000F1F7CE01002E02C0959587950A94E2F77D
:100F100080FF04C0FE240E94950602C00E94920633
:100F20000E94BE06892B11F482E05BC082E390E050
:100F30000E94AB06892B11F483E053C00F5F1F4F53
:100F400008301105D9F680E58A95F1F7FF2019F0F0
:100F50000E94950602C00E9492060E94BE06892B3E
:100F600011F484E03EC082E390E00E94AB06892B3E
:100F700011F485E036C090E59A95F1F70E94950648
:100F8000C2E3D0E00E94A206882341F0209741F0FE
:100F900085E08A95F1F700002197F4CFCD2B11F46D
:100FA00086E01FC082E390E00E94AB06892B11F41B
:100FB00087E017C00E94BE06892B19F0C2E3D0E07B
:100FC00009C088E00EC0209759F095E09A95F1F796
:100FD000000021970E94A2068823A9F3CD2B71F46B
:100FE00089E080933A0180913A01806180933A01CF
:100FF0000E948F060E949506E99A0DC00E948F06F6
:101000000E949506E99ADF91CF911F910F91FF9071
:10101000EF900C9407078FEF9FEFDF91CF911F9117
:101020000F91FF90EF900895CF93DF93809104018B
:1010300090910301981701F1E0910101F0910201F3
:10104000E80FF11D20818F5F909105018923809326
:101050000401C22FD0E08091850380FF0FC01F9252
:101060002F9384E094E09F938F930E9438060F9013
:101070000F900F900F9002C0CFEFDFEFCE01DF9106
:10108000CF9108951F920F920FB60F9211242F93B4
:101090003F934F935F936F937F938F939F93AF9300
:1010A000BF93EF93FF930E94980681118EC08091A9
:1010B000380190913901009781F00E94B7210B9778
:1010C00060F080913701806280933A01109237017D
:1010D0001092360181E0809300010E949F2190933D
:1010E00039018093380180913701893018F48130BB
:1010F00030F012C0893061F18A30B1F146C0809180
:101100003B01813029F40E94A206811105C05DC017
:101110000E94A206811139C0809136018695809384
:1011200036010E94A206882351F080913601806822
:1011300080933601809100018F5F80930001809140
:1011400037018830E9F580913B018130C9F510C045
:101150000E94A20690910001882319F090FF15C00B
:101160002FC090FD12C02CC00E94A206882369F0F7
:10117000809136010E94D206811104C080E48093E0
:101180003A0103C010923A010FC090913A01809148
:101190003701892B80933A0180913A0180933A017B
:1011A000109203011092040110923901109238013B
:1011B000109237011092360181E08093000105C042
:1011C000809137018F5F80933701FF91EF91BF913D
:1011D000AF919F918F917F916F915F914F913F91CF
:1011E0002F910F900FBE0F901F901895CF93C82F7F
:1011F0008DEE0E9442078C2FCF910C944207E82F6E
:10120000E695E695E695EF70F0E0EB5AFE4F4081EB
:10121000282F277081E090E002C0880F991F2A953F
:10122000E2F7242F30E028233923232B11F4842BD9
:1012300080830895E82FE695E695E695EF70F0E057
:10124000EB5AFE4F2081382F377081E090E002C0CA
:10125000880F991F3A95E2F7422F50E0482359230F
:10126000452B19F08095822380830895482F50E004
:10127000FA013397E138F10508F048C0EA5AFF4F08
:101280000C94DD2387E108958FE108958CE508959E
:1012900080E6089582E6089587E2089583E508953B
:1012A0008FE2089589E3089587E308958FE3089511
:1012B00087E408958FE4089586E508958EE50895FE
:1012C0008FE6089580E0089585E608958EE60895F6
:1012D0008FE7089580E3089588E3089580E40895F2
:1012E00088E4089580E5089587E508958FE50895D9
:1012F00088E1089588E0089580E2089580E10895E6
:1013000089E108958DE6089588E208958F7708951C
:101310008FE00895CF93482F50E0FA017C97E8348E
:10132000F105A0F5E952FF4F0C94DD2385E53AC0A5
:101330008AE538C08BE536C08CE534C08DE532C017
:101340008EE530C08FE52EC080E62CC081E62AC035
:1013500082E628C083E626C08FE624C081E722C04B
:1013600082E720C084E71EC085E71CC087E71AC05B
:1013700088E718C08AE716C08CE714C08FE712C050
:1013800080E710C089E70EC08BE70CC0C82F8BE840
:1013900094E09F938F930E9438060F900F908C2FAC
:1013A00001C084E5CF9108950F931F93CF93DF93EE
:1013B0000E949F218C010E941408EC01019631F4D7
:1013C000C8010E94B721883E9340A8F3CE01DF9167
:1013D000CF911F910F910895809185038160809333
:1013E00085030E94F8062E98269A2F98279A2FEFA9
:1013F00089E698E1215080409040E1F700C000006C
:1014000026982798E5E5F1E0119221E0E536F2070C
:10141000D9F70895E82FF0E0EB5AFE4F8081089548
:10142000E5E5F1E0119281E0E536F807D9F7089596
:10143000982F80915201823049F492FB882780F9DD
:1014400090FD826091FD84600C94F6080895CF931E
:10145000DF9380913A01882311F180913A011F9224
:101460008F9384EF94E09F938F930E94380680912E
:101470003A0180750F900F900F900F9071F480914A
:101480005101843051F48EEE94E09F938F930E942B
:101490003806109251010F900F9010923A018091EE
:1014A0005101823089F128F4882351F08130F1F024
:1014B00063C2833009F4CBC0843009F4CFC05CC26E
:1014C00010923B011092520110925401109253015C
:1014D0000E949F219093500180934F0181E080935F
:1014E00051010E94100A0E941D1746C20E94140852
:1014F00080914F01909150010E94B721893E934005
:1015000008F43AC282E0A0C085EF0E94420782EF51
:101510000E9442078F3F4FEF9407A1F08A3F910549
:1015200099F40E94D4098F3F2FEF920781F0D82FB2
:10153000CC270E94D409C82B84EF0E9442079C2F1D
:101540008D2F07C09FEF01C09EEF8FEF02C090E08C
:1015500080E0909353018093540180913A01882355
:1015600081F080913A011F928F9383EE94E09F93D4
:101570008F930E94380610923A010F900F900F90AF
:101580000F90809154018F93809153018F9389ED37
:1015900094E09F938F930E9438068091530190911D
:1015A00054019C0122270F900F900F900F9021154E
:1015B0004BEA340711F482E00CC021153F4B11F4C3
:1015C00083E007C00097B9F38F3F2FEF920721F414
:1015D00081E0809352010DC08F3F910561F783EC4C
:1015E00094E09F938F930E943806109252010F90BF
:1015F0000F90C0915201C13049F48AEB94E09F935F
:101600008F930E943806C0933B011BC0C23019F46F
:1016100081EB94E010C0C33061F482EA94E09F93C0
:101620008F930E94380610923B0188EF0E94420778
:1016300008C084E994E09F938F930E94380610922B
:101640003B010F900F9083E08093510195C10E9460
:1016500095140E94180A84E080935101C0915201B0
:10166000C23009F465C0C33009F417C1C13009F0B4
:1016700083C10E9414088F3F4FEF940709F47CC187
:1016800020914E012230C9F128F4222349F0213063
:10169000C1F04BC02330E9F1243009F43FC045C00C
:1016A000803E910529F0813E910529F482E02EC00B
:1016B000C0934E0161C18038910508F41BC18F773A
:1016C00031C08633910589F124F48A32910539F4C9
:1016D0002CC08A3A910549F1863B910531F1803859
:1016E000910528F40E948A090E94FF081EC08F7786
:1016F0000E948A090E941A0918C08D31910529F0AB
:101700008D39910591F484E001C083E080934E010E
:1017100033C18534910549F485E5ECC085349105E4
:1017200021F485E50E941A0927C110924E0124C1B7
:101730000E9414088F3F2FEF920709F41DC1E0911A
:101740004D014E2F50E04930510508F0A3C0FA0179
:10175000E15EFE4F0C94DD238A3A910509F40CC139
:10176000ACF48338910539F18438910531F1009753
:1017700041F50E94100A8CE794E09F938F930E949A
:10178000380610924D010F900F90F6C0813E9105E2
:1017900081F02CF4803E9105A1F482E072C0803F7C
:1017A000910529F08C3F910509F4E6C00AC081E05B
:1017B00068C084E066C082E001C08FE60E94FF0836
:1017C00069C080389105D0F30E94100A80E794E048
:1017D0009F938F930E9438060F900F905BC08935BE
:1017E000910509F457C0803F910521F082319105A0
:1017F00019F450C083E045C08038910518F40E9468
:101800003609DCCF0E94100A86E694E0E1CF8338E7
:10181000910529F08438910521F48FE639C082E0E2
:1018200037C080389105A0F10E94100A8CE594E041
:10183000CFCF8231910571F18935910559F1803809
:10184000910518F40E94360923C00E94100A8FE403
:1018500094E0BECF8431910529F0803F9105D1F409
:1018600086E00FC085E00DC08737910599F480E0D0
:10187000A5CF449779F487E004C0803F910551F4E7
:1018800088E080934D0178C08737910519F480E096
:101890000E941A0910924D016FC00E9414088F3FD8
:1018A0004FEF940709F468C020914C01222319F0EE
:1018B0002130B1F161C084389105D9F03CF4009732
:1018C00059F083389105C9F482E014C0803F910536
:1018D00061F08F3F910589F49F938F9383E494E0A7
:1018E0009F938F930E94380632C081E080934C0111
:1018F00043C08FE70E94FF083FC08038910518F46D
:101900000E94FF082EC09F938F9387E394E09F93DC
:101910008F930E9438060F900F900F900F9021C068
:1019200083389105C9F01CF4009739F01DC0843844
:101930009105A1F08F3F9105B9F49F938F9388E2B1
:1019400094E09F938F930E94380610924C010F9061
:101950000F900F900F9010C082E001C08FE70E949F
:101960001A0910924C0108C080389105C0F39F936A
:101970008F9389E194E0CBCF81E0DF91CF910895FF
:101980008091890208950895CF93DF9300D01F922C
:10199000CDB7DEB720918F03243021F523E02983D2
:1019A0009B838A8382E08093E9008FEF9091E80027
:1019B000815095FD06C095ED9A95F1F700008111D3
:1019C000F5CF8091E80085FF0DC040E050E063E076
:1019D00070E0CE0101960E9444108091E8008E775D
:1019E0008093E8000F900F900F90DF91CF910895B2
:1019F000CF93DF9300D01F92CDB7DEB720918F0336
:101A0000243029F522E02983805891099B838A8319
:101A10002093E9008FEF9091E800815095FD06C07A
:101A200095ED9A95F1F700008111F5CF8091E800CE
:101A300085FF0DC040E050E063E070E0CE0101960C
:101A40000E9444108091E8008E778093E8000F9008
:101A50000F900F90DF91CF910895CF93DF93EC011A
:101A600090918F03943009F048C08091150188232C
:101A7000D9F0809116018823B9F09093E90081E8AC
:101A8000815049F09091E80095FD05C09AE29A9541
:101A9000F1F700C0F5CF8091E80085FF2EC040E04F
:101AA00050E060E270E019C081E08093E90081E8D5
:101AB000815059F09091E80095FD07C0EFE3F1E007
:101AC0003197F1F700C00000F3CF8091E80085FF67
:101AD00014C040E050E068E070E0CE010E94441085
:101AE0008091E8008E778093E80080E2FE01A9E60D
:101AF000B2E001900D928A95E1F7DF91CF910895C0
:101B0000CF93C0916701C1110BC00E94AB21643C0F
:101B100079408105910520F081E080936701C1E063
:101B20008C2FCF910895CF93C82F0E94800D8823CA
:101B300009F448C00FB607FE45C080918F0384307A
:101B400009F040C08091E9008F702091EC00922F45
:101B5000917020FD90E8892B93E09093E90090919B
:101B6000EB0090FF2CC09091EE0097FF28C0909161
:101B7000090120910801291709F447C02091E800C4
:101B800025FF1DC0E0910601F0910701E90FF11D4D
:101B900030819F5F20910A01922390930901309335
:101BA000F1009091E80095FDE2CF9091E80090FF60
:101BB000DECF9091E8009E779093E800D8CF8F70A9
:101BC0008093E9008091080190E0AC014F5F5F4F86
:101BD00030910A01232F30E024233523409109015D
:101BE00050E024173507D1F020910601309107010C
:101BF000F901E80FF91FC083809108018F5F909170
:101C00000A0189238093080109C09091E80095FF9B
:101C1000D6CFC093F1008F708093E90080E0CF9120
:101C2000089580918E03811109C00E94D7110E94EE
:101C300034128091E20084608093E2000895109253
:101C40008E0308950895089542E061EC81E00E94BA
:101C5000501142E061EC82E00E94501142E261ECDE
:101C600083E00E94501142E261EC84E00C94501138
:101C700080919103833009F455C030F4813071F0C4
:101C8000823009F48EC008958A3009F47AC08B300E
:101C900009F460C0893009F09CC020C08091900395
:101CA000813A09F096C08091E800877F8093E80030
:101CB0008091940390919503892B21F460E289E649
:101CC00092E003C060E080E090E070E00E9491103C
:101CD0008091E8008B778093E800089580919003CD
:101CE000813209F076C0809194039091950300971A
:101CF00019F0039709F06DC08091E800877F809309
:101D0000E8008091E80082FD05C080918F03811179
:101D1000F8CF5FC08091F100809389028091E80044
:101D20008B7753C080919003813A09F052C0809123
:101D3000940390919503892B09F04BC08091E800A2
:101D4000877F8093E8008091E80080FFFCCF80913E
:101D5000150136C0809190038132D9F580919403AA
:101D600090919503892BA9F58091E800877F809356
:101D7000E8000E94851180919203809315010C94D4
:101D80001D1780919003813221F58091E800877FB3
:101D90008093E8000E9485118091930380938A02CA
:101DA000089580919003813AA1F48091E800877FA3
:101DB0008093E8008091E80080FFFCCF80918A0248
:101DC0008093F1008091E8008E778093E8000C9476
:101DD000851108958091890280936801109289028B
:101DE0000E94100A0C941D170C94EA0E0E944C21BC
:101DF00080918D03882329F00E94592181110C9430
:101E00002E1008950E946D218091680180938902AF
:101E100008950C94020F08950C940B0F0C940B0F63
:101E2000CF9384B7877F84BF0FB6F894A89580912D
:101E30006000886180936000109260000FBE90E0A7
:101E400080E80FB6F89480936100909361000FBE14
:101E500083E99DE00E941F218BE091E00E94901495
:101E600083E295E00E949F050E940E0F0E94441598
:101E70000E94D7110E9434128091E2008460809306
:101E8000E20078940E94461580918F03843029F0F7
:101E90000E9475140E940B0FF7CF81E195E00E941C
:101EA0009F050E940C0F8FEF94E00E949F05C3E0F6
:101EB00080918F03853019F40E94F60EF9CF0E94AD
:101EC0004A152091E4003091E500809165019091E0
:101ED00066012817390709F468C08091E4009091E1
:101EE000E50090936601809365010E94800D882330
:101EF00009F45BC080918F03843009F056C0809153
:101F0000E9008F702091EC00922F917020FD90E8F5
:101F1000892BC093E9009091EB0090FF43C0909112
:101F2000EE0097FF3FC09091090120910801291709
:101F300009F12091E80025FF1DC0E0910601F09114
:101F40000701E90FF11D30819F5F20910A01922363
:101F5000909309013093F1009091E80095FDE3CF53
:101F60009091E80090FFDFCF9091E8009E779093EA
:101F7000E800D9CF9091F3002091F20030E0392BA6
:101F8000232B81F09091E80090FF0CC09091E80025
:101F900095FF03C01092F100F9CF9091E8009E7771
:101FA0009093E8008F708093E9000E94751480CFB1
:101FB000292F332723303105C9F060F42130310552
:101FC00081F02230310509F041C084E790E023E838
:101FD00035E040C021323105E1F02232310531F1E6
:101FE00035C082E190E027EF35E034C09927813099
:101FF000910549F028F0029749F5E9E3F5E005C0BD
:10200000EFE7F5E002C0EFE6F5E0849190E09F0194
:1020100021C06430D8F4E62FF0E0EE0FFF1FEB5D37
:10202000FE4F2081318189E090E014C0643070F46B
:1020300070E0FB01EE0FFF1FE35EFE4F2081318158
:10204000FB01E75EFE4F808190E004C080E090E0FD
:1020500020E030E0FA0131832083089580E189BDDA
:1020600082E189BD09B400FEFDCF8091D8008F7D4B
:102070008093D8008091E00082608093E00080919E
:10208000E00081FDFCCF0895CF92DF92EF92FF92A6
:102090000F931F93CF93DF93EC018B017A010E9482
:1020A000A411811135C0E114F10439F0F7018081E8
:1020B0009181081B190BC80FD91FC12CD12C0115F8
:1020C000110529F18091E80085FD18C08091E80094
:1020D0008E778093E8000E947514E114F10449F0B2
:1020E000F70180819181C80ED91ED182C08285E01E
:1020F0000FC00E94A411882311F30AC08991809314
:10210000F10001501109FFEFCF1ADF0AD8CF80E0AC
:10211000DF91CF911F910F91FF90EF90DF90CF90C3
:10212000089520919603309197032617370748F0BA
:102130006115710539F42091E8002E772093E800AD
:1021400001C0B901FC0120E06115710579F18091B0
:102150008F038823F1F18530F1F18091E80083FD50
:102160003CC08091E80082FD2EC08091E80080FF95
:10217000EBCF2091F3008091F20090E0922B61155B
:10218000710551F08830910538F421912093F100C8
:10219000615071090196F3CF21E0089709F020E022
:1021A0008091E8008E778093E800CECF2111CFCFC9
:1021B0000AC080918F03882361F0853061F080919F
:1021C000E80083FD0AC08091E80082FFF2CF80E042
:1021D000089582E0089583E0089581E008952091B4
:1021E0009603309197032617370748F0611571055C
:1021F00039F42091E8002E772093E80001C0B9015E
:10220000FC0120E06115710591F180918F03882315
:1022100009F440C0853009F43FC08091E80083FD97
:102220003DC08091E80082FD2FC08091E80080FFD2
:10223000E9CF2091F3008091F20090E0922B61159C
:10224000710559F08830910540F424912093F100F4
:102250003196615071090196F2CF21E0089709F09B
:1022600020E08091E8008E778093E800CBCF2111A9
:10227000CCCF0AC080918F03882361F0853061F054
:102280008091E80083FD0AC08091E80082FFF2CFD0
:1022900080E0089582E0089583E0089581E0089544
:1022A000982F973068F59093E900981739F070915E
:1022B000EC002091ED005091F00003C0242F762F08
:1022C00050E021FD02C09F5FECCF3091EB003E7FDC
:1022D0003093EB003091ED003D7F3093ED00309175
:1022E000EB0031603093EB007093EC002093ED0035
:1022F0005093F0002091EE0027FDE5CF80E0089597
:102300008F708093E90081E008958091900387FFAA
:1023100011C08091E80082FD05C080918F0381117A
:10232000F8CF11C08091E8008B770BC080918F03AC
:10233000882349F08091E80080FFF8CF8091E80081
:102340008E778093E80008952091E4003091E500B5
:1023500095E64091EC00842F817040FF23C080916E
:10236000E80080FD1DC080918F03882399F085309F
:1023700099F08091EB0085FD11C04091E4005091EF
:10238000E5002417350729F3915011F09A01E1CFA8
:1023900084E0089582E0089583E0089581E008953F
:1023A00080E008954091E80042FFDDCF08950E944B
:1023B00045120E944D12E0EEF0E080818160808342
:1023C000E8EDF0E080818F77808319BCA7EDB0E065
:1023D0008C918E7F8C9380818F7E808310928E0370
:1023E00008950F931F93CF93DF930E9445120E948D
:1023F0004D12C8EDD0E088818F778883888180680E
:10240000888388818F7D888319BC10928F031092F6
:102410008B0310928D0310928C0300EE10E0F801F4
:1024200080818B7F808388818160888342E060E047
:1024300080E00E945011E1EEF0E080818E7F808389
:10244000E2EEF0E08081816080838081886080831B
:10245000F80180818E7F8083888180618883DF910D
:10246000CF911F910F910895E8EDF0E080818F7E6C
:102470008083E7EDF0E080818160808384E082BF2B
:1024800081E080938E030C94F111E8EDF0E08081FF
:102490008E7F80831092E20008951092DA001092ED
:1024A000E10008951F920F920FB60F9211242F93FF
:1024B0003F934F935F936F937F938F939F93AF93CC
:1024C000BF93EF93FF938091E10082FF0BC0809157
:1024D000E20082FF07C08091E1008B7F8093E100E2
:1024E0000E94230E8091DA0080FF1FC08091D800E7
:1024F00080FF1BC08091DA008E7F8093DA0080918C
:10250000D90080FF0DC080E189BD82E189BD09B499
:1025100000FEFDCF81E080938F030E94110E05C065
:1025200019BC10928F030E941F0E8091E10080FF62
:1025300019C08091E20080FF15C08091E2008E7F7B
:102540008093E2008091E20080618093E2008091BC
:10255000D80080628093D80019BC85E080938F03F7
:102560000E94F40E8091E10084FF30C08091E2006F
:1025700084FF2CC080E189BD82E189BD09B400FEE1
:10258000FDCF8091D8008F7D8093D8008091E100AD
:102590008F7E8093E1008091E2008F7E8093E20045
:1025A0008091E20081608093E20080918B03882318
:1025B00011F084E007C08091E30087FD02C081E054
:1025C00001C083E080938F030E94090F8091E10096
:1025D00083FF24C08091E20083FF20C08091E1004E
:1025E000877F8093E10082E080938F0310928B03BA
:1025F0008091E1008E7F8093E1008091E2008E7FE8
:102600008093E2008091E20080618093E20042E0EA
:1026100060E080E00E9450110E94220EFF91EF9135
:10262000BF91AF919F918F917F916F915F914F91EA
:102630003F912F910F900FBE0F901F9018951F93F1
:10264000CF93DF93CDB7DEB7AA970FB6F894DEBF6E
:102650000FBECDBFE0E9F3E08091F100819323E06C
:10266000E839F207C9F70E94380E8091E80083FF2D
:1026700024C18091900390919103492F50E04A30FA
:10268000510508F01AC1FA01E85DFE4F0C94DD23F4
:10269000803881F0823809F010C1809194038F70E6
:1026A0008093E9008091EB0085FB882780F91092E8
:1026B000E90006C080918C0390918D039111826096
:1026C0009091E800977F9093E8008093F10010923A
:1026D000F100C8C0282F2D7F09F0EFC0882319F022
:1026E000823061F0EAC080919203813009F0E5C048
:1026F000933009F080E080938D032BC0809192038A
:10270000811127C0809194038F7009F4D6C0809303
:10271000E9002091EB0020FF1CC0933021F4809150
:10272000EB00806214C09091EB0090619093EB00FD
:1027300021E030E0A90102C0440F551F8A95E2F75D
:102740004093EA001092EA008091EB008860809349
:10275000EB001092E9008091E800877F86C081112C
:10276000ACC0109192031F778091E3008078812B99
:102770008093E3008091E800877F8093E8000E94C7
:1027800085118091E80080FFFCCF8091E300806894
:102790008093E300111102C082E001C083E08093C6
:1027A0008F038BC08058823008F087C080919203DD
:1027B000909193038C3D53E0950779F583E08A83EC
:1027C0008AE289834FB7F894DE01139620E03EE059
:1027D00051E2E32FF0E050935700E49120FF03C053
:1027E000E295EF703F5FEF708E2F90E0EA3010F0CF
:1027F000C79601C0C0968D939D932F5F243149F7F2
:102800004FBF8091E800877F8093E8006AE270E024
:10281000CE0101960E94911014C0AE014F5F5F4F30
:10282000609194030E94D80FBC01892B09F445C024
:102830009091E800977F9093E80089819A810E94A7
:10284000EF108091E8008B778093E80036C08038E5
:10285000A1F58091E800877F8093E80080918B0349
:102860008093F1008091E8008E778093E8000E94C9
:10287000851123C0811121C080919203909193030F
:1028800099270297D4F48091E800877F8093E8002D
:102890008091920380938B030E94851180918B031A
:1028A000811106C08091E30087FD02C081E001C074
:1028B00084E080938F030E94240E8091E80083FFC0
:1028C0000AC08091E800877F8093E8008091EB0048
:1028D00080628093EB00AA960FB6F894DEBF0FBE1D
:1028E000CDBFDF91CF911F910895CF9380918F033A
:1028F0008823A1F0C091E900CF709091EC00892F5E
:10290000817090FD80E8C82B1092E9008091E8006A
:1029100083FD0E941F13CF70C093E900CF910895EB
:102920009093900280938F020895E0918F02F0912E
:102930009002309721F00190F081E02D099480E021
:102940000895EF92FF920F931F93CF93DF93E0913F
:102950008F02F09190023097B1F18C010280F381E7
:10296000E02D09958091850382FF2DC080FF04C072
:1029700080E097E00E949F05E80110E28AEFE82ED0
:1029800086E0F82E8091850380FF0BC088811F921E
:102990008F93FF92EF920E9438060F900F900F9046
:1029A0000F90115021961111EDCF8091850380FF7A
:1029B0000AC088EF96E0DF91CF911F910F91FF90B1
:1029C000EF900C949F05DF91CF911F910F91FF9095
:1029D000EF900895CF93DF9320918D0230918E0276
:1029E0002817390709F190938E0280938D02E091A8
:1029F0008F02F09190023097B9F0EC010680F781D8
:102A0000E02D09958091850382FF0EC080FF0CC0E8
:102A1000DF93CF938AEE96E09F938F930E943806C0
:102A20000F900F900F900F90DF91CF910895CF935B
:102A3000DF9320918B0230918C022817390709F11E
:102A400090938C0280938B02E0918F02F091900220
:102A50003097B9F0EC010084F185E02D0995809163
:102A6000850382FF0EC080FF0CC0DF93CF938AEDF9
:102A700096E09F938F930E9438060F900F900F90CF
:102A80000F90DF91CF9108950C94ED150E9496213F
:102A90000C94EC09BF92CF92DF92EF92FF920F93CA
:102AA0001F93CF93DF9300D000D01F92CDB7DEB736
:102AB0000E94270A02E912E0F12C8F2D0E940A0AD7
:102AC000B82EF801C080C82639F4F3940F5F1F4F69
:102AD000F0E1FF12F2CF30C08091850381FD0E94AA
:102AE000EE15D12CEE24E3948C2D8E21F9F0D982B1
:102AF000FA8291E08B2D8E2109F490E09B830E9455
:102B00009F218160782F9D838C8349815A816B81BD
:102B10008D810E94241649815A816B817C818D812F
:102B20000E943721F80180818E258083D394EE0C9A
:102B3000F8E0DF12D9CFC9CF8FEF89838A831B8258
:102B40000E949F218160782F9D838C8349815A81C7
:102B50006B818D810E9424160E9436210E9495145B
:102B600090919102891741F10E94951480939102EE
:102B70009091850392FF0EC090FF0CC01F928F931F
:102B80008BE097E09F938F930E9438060F900F90F1
:102B90000F900F90809191020F900F900F900F90D7
:102BA0000F90DF91CF911F910F91FF90EF90DF90E9
:102BB000CF90BF900C9448210F900F900F900F90E2
:102BC0000F90DF91CF911F910F91FF90EF90DF90C9
:102BD000CF90BF9008950C94180A0895EF92FF9239
:102BE0000F931F93CF93DF9384E297E00E949F059A
:102BF000C0E0D0E08DE2E82E81E0F82E06E117E09B
:102C00008C2F0E940A0A0E942421FF92EF921F92A9
:102C10008F93DF93CF931F930F930E9438062196D3
:102C20008DB79EB708960FB6F8949EBF0FBE8DBFA6
:102C3000C031D10529F7DF91CF911F910F91FF90FE
:102C4000EF90089508950895CF93DF93CDB7DEB741
:102C50002B970FB6F894DEBF0FBECDBF942F4F83D6
:102C6000252F588769877A878B874A855B85452B0F
:102C700031F02F3F31F481E09F3F19F403C081E030
:102C800001C080E080FD07C04F81588569857A8545
:102C90008B850E943721DE01119686E0FD0111929D
:102CA0008A95E9F785E0FE01379601900D928A95A5
:102CB000E1F749815A816B817C818D819E810E94DF
:102CC000321D2B960FB6F894DEBF0FBECDBFDF913D
:102CD000CF910895CF93882309F465C0C82F8CEF56
:102CE0008C0F813A20F080E58C0F8E3248F48C2FC7
:102CF0000E948A23811157C08C2F0E941A200CC079
:102D000080E28C0F883058F4C77081E001C0880FD2
:102D1000CA95EAF70E94BF20CF910C94F9208BE569
:102D20008C0F833078F4C53A29F0C63A31F083E845
:102D300090E005C081E890E002C082E890E0CF9189
:102D40000C94EA1488E58C0F853168F5C83A89F04F
:102D5000C93A91F0CA3A99F0CB3AA1F0CC3AA9F02D
:102D6000CD3AB1F0CE3AB9F0CF3AC1F080E090E080
:102D700017C082EE90E014C089EE90E011C08AEE98
:102D800090E00EC085EB90E00BC086EB90E008C0B1
:102D900083EB90E005C084EB90E002C087EB90E00D
:102DA000CF910C941715CF910895882349F19CEF8A
:102DB000980F913A20F090E5980F9E3218F40E94F7
:102DC0006A200DC090E2980F983058F4877091E017
:102DD00001C0990F8A95EAF7892F0E94C5200C94AB
:102DE000F9209BE5980F933020F480E090E00C945C
:102DF000EA14885A853120F480E090E00C9417158D
:102E00000895882321F00E94BF200C94F920089592
:102E1000882321F00E94C5200C94F92008950E9477
:102E2000DF200E94AE200E94F92080E090E00E9406
:102E3000EA1480E090E00C9417150E94CF200C94C7
:102E40000F17CF92DF92EF92FF920F931F93CF93C2
:102E5000DF9300D000D01F92CDB7DEB76C010E9487
:102E60004A218111EAC285E0F601DE011196019046
:102E70000D928A95E1F7F6014081518123813481D9
:102E80002115310531F05F3F31F481E04F3F19F4F6
:102E900003C081E001C080E080FDCFC2F601F28076
:102EA000E580E2948FE0E82249835A83FB82722F07
:102EB0003D832C836F2D8D810E94961F8C010E9473
:102EC000951F0E94851EE12FE295EF708E2F90E0F6
:102ED000FC01EE5CFE4F0C94DD23812F807F1F7080
:102EE000882311F01295107FFF2049F0112309F477
:102EF0003BC2812F0E94D2200E94F92035C2802F30
:102F00000E94D516112309F498C2812F0E94D8205F
:102F10000F900F900F900F900F90DF91CF911F9116
:102F20000F91FF90EF90DF90CF900C94F920812FBC
:102F3000807F1F70803211F01295107F002319F0EE
:102F4000013009F12BC0FF20A9F0EE2059F1F1E08A
:102F5000812FEF1228C00F900F900F900F900F90BD
:102F6000DF91CF911F910F91FF90EF90DF90CF9065
:102F70000C94E220EE2021F021E0E21609F45DC27B
:102F80000E94E5202DC0FF20E9F085E08E1508F4B1
:102F900054C20E94BC20812329F022C0FF20F1F0FE
:102FA000E11015C0812F0F900F900F900F900F9090
:102FB000DF91CF911F910F91FF90EF90DF90CF9015
:102FC0000C94011794E09E1508F437C209C0F6016D
:102FD000858180FFC9C18F708583E4CFE110D7C19F
:102FE000812F4AC1812F86958695837019F0813093
:102FF000B9F023C2FF2019F0C801937002C080E02D
:1030000090E00F900F900F900F900F90DF91CF9165
:103010001F910F91FF90EF90DF90CF900C94EA14E6
:10302000FF2019F0C801937002C080E090E00F907B
:103030000F900F900F900F90DF91CF911F910F91F4
:10304000FF90EF90DF90CF900C941715812F837035
:1030500009F070C0F110F1C1202F2295269527703C
:10306000220F220F602F6F70862F90E0A0E0B0E05B
:103070006C017D01022E04C0CC0CDD1CEE1CFF1C7B
:103080000A94D2F704FF12C08FE090E0A0E0B0E015
:1030900004C0880F991FAA1FBB1F2A95D2F7BC0135
:1030A000CD01609570958095909503C060E070E0CB
:1030B000CB011695169513701230B1F040F56C29BE
:1030C0007D298E299F29113031F10F900F900F909B
:1030D0000F900F90DF91CF911F910F91FF90EF9084
:1030E000DF90CF900C94AA1E6C297D298E299F29F0
:1030F0000F900F900F900F900F90DF91CF911F9135
:103100000F91FF90EF90DF90CF900C94C41E0E941F
:10311000AA1EC701B6010F900F900F900F900F904D
:10312000DF91CF911F910F91FF90EF90DF90CF90A3
:103130000C94901EFF2019F0812F817001C086959C
:10314000882309F47AC1202F229526952770220F13
:10315000220F602F6F70862F90E0A0E0B0E06C012E
:103160007D01022E04C0CC0CDD1CEE1CFF1C0A9459
:10317000D2F704FF12C08FE090E0A0E0B0E004C0FE
:10318000880F991FAA1FBB1F2A95D2F7BC01CD013A
:10319000609570958095909503C060E070E0CB01DC
:1031A0001695169513701230B1F040F56C297D29F3
:1031B0008E299F29113031F10F900F900F900F90B1
:1031C0000F90DF91CF911F910F91FF90EF90DF90C3
:1031D000CF900C94711F6C297D298E299F290F9007
:1031E0000F900F900F900F90DF91CF911F910F9143
:1031F000FF90EF90DF90CF900C94831F0E94711F7F
:10320000C701B6010F900F900F900F900F90DF91B4
:10321000CF911F910F91FF90EF90DF90CF900C9482
:103220005F1F003FC1F128F480E4800F803250F02E
:1032300096C0023F09F45EC008F449C0033F09F498
:103240006CC08DC0F02FF071EF2E812F8F71FF2099
:1032500051F00E94F81E802FEE2019F08295807F99
:10326000A2CE8F70A0CE0E94191F802FEE2019F0E1
:103270008295807F01C08F700F900F900F900F90FC
:103280000F90DF91CF911F910F91FF90EF90DF9002
:10329000CF900C940817FF20A9F024E02E1508F415
:1032A000CCC0812F8F710F900F900F900F900F90C7
:1032B000DF91CF911F910F91FF90EF90DF90CF9012
:1032C0000C943E1F85E08E1508F4B7C0EACFFF20AE
:1032D00099F0812F8F710F900F900F900F900F909A
:1032E000DF91CF911F910F91FF90EF90DF90CF90E2
:1032F0000C94F81EFF2069F3812F8F710F900F90AF
:103300000F900F900F90DF91CF911F910F91FF9031
:10331000EF90DF90CF900C94191FFF2089F0812F40
:103320008F710F900F900F900F900F90DF91CF91B2
:103330001F910F91FF90EF90DF90CF900C94E31EC0
:103340000F900F900F900F900F90DF91CF911F91E2
:103350000F91FF90EF90DF90CF900C94DE1EFF2036
:1033600099F0EE2009F4B5CF802F0F900F900F90B9
:103370000F900F90DF91CF911F910F91FF90EF90E1
:10338000DF90CF900C946A16EE2009F4B5CF802F11
:103390000F900F900F900F900F90DF91CF911F9192
:1033A0000F91FF90EF90DF90CF900C94D516412FA6
:1033B0004F70602FC6010E9425220F900F900F9032
:1033C0000F900F90DF91CF911F910F91FF90EF9091
:1033D000DF90CF900C94E01D01112FC0FF2069F108
:1033E0000E941D179FEFE0E7F2E09150E040F040AF
:1033F000E1F700C000000F900F900F900F900F901A
:10340000DF91CF911F910F91FF90EF90DF90CF90C0
:103410000C940622412F4F70602FC6010F900F9021
:103420000F900F900F90DF91CF911F910F91FF9010
:10343000EF90DF90CF900C9428220F900F900F9078
:103440000F900F90DF91CF911F910F91FF90EF9010
:10345000DF90CF9008951F93CF93DF9300D000D0DB
:103460001F92CDB7DEB7942F4983252F5A836B83E4
:103470007C838D834C815D81452B31F02F3F31F46E
:1034800081E09F3F19F403C081E001C080E0182F64
:10349000117080FD31C049815A816B817C818D81A1
:1034A0000E94961F292F22952F702C3030F42A303D
:1034B000A0F42250223030F022C02C30C9F02F303E
:1034C000B9F01DC0853A28F48430C0F4823028F465
:1034D00015C090E2980F983088F0883E30F4803E16
:1034E00068F48450813A58F409C0803F41F406C022
:1034F00093FB112710F903C010E001C011E0812FE8
:103500000F900F900F900F900F90DF91CF911F9120
:103510000895CF93DF9300D000D01F92CDB7DEB7D0
:103520000F900F900F900F900F90DF91CF91089513
:10353000CF93DF9300D000D000D0CDB7DEB7269672
:103540000FB6F894DEBF0FBECDBFDF91CF910895C7
:103550001F93CF93DF93C091A20216E08091A30244
:10356000C81799F0D0E01C9FF0011D9FF00D1124A9
:10357000EC55FD4F40815181628173818481958139
:103580000E94981A2196C770E9CFDF91CF911F91C1
:1035900008954091D4025091D5026091D602709165
:1035A000D7028091D8029091D9020C94981ACF93A7
:1035B0008091D90282958F7009F05FC08091D60208
:1035C000882309F45AC08091A202B091A30270919D
:1035D000D402A091D5024091D7025091D80291E037
:1035E0007F3F09F090E0692FC6E08B1709F445C0D2
:1035F0004115510521F0AF3F21F020E003C021E04B
:1036000001C0262F90E020FD35C0C89FF001C99F62
:10361000F00D1124EC55FD4F21812A132BC0208180
:10362000271328C02281211125C02381348124172A
:10363000350710F421503109241B350B283C310586
:10364000C8F42091D9022F7020612093D90226E07E
:10365000289FF001299FF00D1124E755FD4F80812F
:103660008F708061808384ED92E00E942117CF915A
:103670000C94A81A01968770B8CFCF910895AF9295
:10368000BF92CF92DF92EF92FF920F931F93CF934F
:10369000DF93CDB7DEB761970FB6F894DEBF0FBEEC
:1036A000CDBF7C0185E0F701DE011D9601900D92F2
:1036B0008A95E1F7D7014C9111965C91119712967A
:1036C000DC90129713960D911C9114973091D402AF
:1036D0006091D5028091D7029091D802009731F085
:1036E0006F3F31F421E03F3F19F403C021E001C0F6
:1036F00020E0B22FB170BB2E20FD6EC1A090D6028B
:10370000AA2009F4CCC02091D9020817190728F083
:10371000F801E81BF90BCF0104C080959095800F4C
:10372000911FCC24C394883C910580F0C12C207F4C
:1037300009F0A1C0702F198B088B6D2D89890E940B
:10374000891A84ED92E00E942117BDC0822F807FEC
:1037500009F056C0561315C0431313C0CD2CD11019
:1037600010C02F7020612093D9020E94C91A84EDE5
:1037700092E00E9421178091D902D70115968C936F
:103780005FC10115110531F05F3F31F481E04F3F1A
:1037900019F403C081E001C080E080FD03C081E036
:1037A0008D2502C080E090E0B82FB170CB2E80FF55
:1037B0001CC08091A2022091A30236E0821709F476
:1037C0001CC190E0389FF001399FF00D1124EC5599
:1037D000FD4F6181561306C06081461303C06281AC
:1037E000D61203C001968770E9CFCD2CDD2009F4F5
:1037F00027C18091D90281608093D902C12C20C158
:10380000561308C0431306C0D11004C08091D902DA
:10381000D701B6C04D875E87DF86702F198B088B66
:103820006D2D89890E942B1A882399F1DD2089F159
:103830002091D902822F82958F7090E0029774F0C8
:103840008091D4029091D50298878F8319861B8727
:103850000A872C87CE0107960E94211786E0F70180
:10386000A4EDB2E001900D928A95E1F70E94D71A7B
:103870000E94C91A11C0561781F14D875E87DF86F5
:10388000702F198B088B6D2D89890E942B1A81113D
:1038900038C0C7010E942117CC24C394D1C0081797
:1038A000190708F446C0F801E81BF90BCF01883C62
:1038B000910508F443C0C12C702F198B088B6D2D16
:1038C00089890E94891AE4EDF2E086E0DF011D9209
:1038D0008A95E9F70E94C91AB3C04313CECFD1101D
:1038E000CCCF8091D902F7018583C7010E942117AF
:1038F00086E0E4EDF2E0DF011D928A95E9F7CA2C3B
:103900009FC0DD2031F22091D902822F82958F70E5
:1039100090E002970CF4A2CF8091D4029091D5024E
:103920009A8389831B821D830C832E83CE0101968B
:1039300093CF80959095800F911FB9CFCD2CDD202E
:1039400009F4A7CF561333C0431331C02091D902D5
:1039500020FD24C0822F82958F70482F50E04115A2
:103960005105E1F0D70115962C9315974F3051056D
:1039700049F08F5F982F9295907F822F8F70892BBF
:1039800015968C93C7010E94211786E0F701A4EDDC
:10399000B2E001900D928A95E1F79CCF86E0F701A5
:1039A000A4EDB2E001900D928A95E1F749C04D87F0
:1039B0005E87DF86702F198B088B6D2D89890E9499
:1039C0002B1A81114BCF8091D90281608093D9024B
:1039D000C7010E94211734C0DD2009F45ACF4D875A
:1039E0005E87DF86702F198B088B6D2D89890E9469
:1039F0002B1A882309F44DCF31CF702F198B088BE8
:103A00006D2D89890E94961F292F22952F702230B3
:103A100028F49F7039F0811105C00BC0243028F4C0
:103A20009F7049F4805E883020F0C7010E94211702
:103A3000BC2CCB2C05C0F7019581907F99F7F9CF6D
:103A40008C2D61960FB6F894DEBF0FBECDBFDF910F
:103A5000CF911F910F91FF90EF90DF90CF90BF908B
:103A6000AF9008951F93CF93DF93CDB7DEB72C9718
:103A70000FB6F894DEBF0FBECDBF4F83588769875E
:103A80007A878B879C87CE0107960E943F1B8823ED
:103A9000D1F09F8188852A853B85232B31F08F3F8C
:103AA00031F481E09F3F19F403C081E001C080E060
:103AB00080FD47C04F81588569857A858B859C85B7
:103AC0000E94981A3EC086E0FE013796DE011196EC
:103AD00001900D928A95E1F7FF81E8856A857B85E3
:103AE0006115710531F0EF3F31F481E0FF3F19F4CA
:103AF00003C081E001C080E080FD23C02091A302CB
:103B000030E0C9010196877099274091A20250E0E8
:103B100084179507F1F1F983EA837D836C8396E03E
:103B2000929FD001939FB00D1124AC55BD4FFE0163
:103B3000319601900D929A95E1F78093A3020E942D
:103B4000A81A16E08091A2029091A302891771F140
:103B5000189FC00111248C559D4F0E943F1B882344
:103B600029F1E091A2021E9FF0011124EC55FD4FB6
:103B70004081518162817381848195810E94981A6C
:103B80008091A20290E00196877099278093A2020B
:103B9000D9CF0E941D171092A3021092A202E4ED49
:103BA000F2E086E0DF011D928A95E9F72C960FB6C8
:103BB000F894DEBF0FBECDBFDF91CF911F91089566
:103BC000DF92EF92FF920F931F93CF93DF93FC014D
:103BD000892B09F488C0E12CF12CDD24D394EF016A
:103BE00021968491853709F460C058F4843708F031
:103BF0004EC0843008F068C08130D1F0823071F15D
:103C000072C0883709F45BC050F4863709F453C09A
:103C1000873709F068C08E2D0E94CC2052C09CE7E7
:103C2000980F903708F05FC08F770E94D5164EC06E
:103C30008F010E5F1F4FFE01849190E2980F983024
:103C400050F48770FD2D01C0FF0F8A95EAF78F2F82
:103C50000E94D22015C00E946A1614C08F010E5F08
:103C60001F4FFE01849190E2980F983068F487709E
:103C7000FD2D01C0FF0F8A95EAF78F2F0E94D820F3
:103C80000E94F920E80122C00E94D516FBCFCF0187
:103C90000296FE01C491CC2361F0EFE9FFE0319779
:103CA000F1F700C00000C150F6CFCF010296FE012F
:103CB000F490EC010BC00E94BC20E82E07C00E94CB
:103CC000CF200E94F92002C00E946A168F2D8823FF
:103CD00041F0EFE9FFE03197F1F700C000008150BB
:103CE000F6CFFE017CCFDF91CF911F910F91FF9016
:103CF000EF90DF90089560935A0370935B03809375
:103D00005C0390935D030C944721089560935E03D8
:103D100070935F0380936003909361030C9446213A
:103D20000F931F9300915E0310915F032091600336
:103D300030916103602B712B822B932B60935E0378
:103D400070935F0380936003909361031F910F91C1
:103D50000C9446210F931F9300915E0310915F0313
:103D600020916003309161036023712382239323A8
:103D700060935E0370935F0380936003909361038D
:103D80001F910F910C9446210F931F9300915E0396
:103D900010915F03209160033091610360277127C8
:103DA0008227932760935E0370935F038093600381
:103DB000909361031F910F910C94462160E070E095
:103DC000CB010C947B1E0F931F9341E050E060E009
:103DD00070E08A019B0104C0000F111F221F331FD6
:103DE0008A95D2F7C901B8011F910F910C947B1EDF
:103DF0000F931F9341E050E060E070E004C0440F77
:103E0000551F661F771F8A95D2F780915A039091AC
:103E10005B03A0915C03B0915D038A019B01082BB9
:103E2000192B2A2B3B2BC901B8011F910F910C9420
:103E30007B1E0F931F9341E050E060E070E004C0F0
:103E4000440F551F661F771F8A95D2F740955095EE
:103E50006095709580915A0390915B03A0915C03EB
:103E6000B0915D038A019B01082319232A233B2378
:103E7000C901B8011F910F910C947B1E0F931F93E2
:103E800041E050E060E070E004C0440F551F661F41
:103E9000771F8A95D2F780915A0390915B03A09186
:103EA0005C03B0915D038A019B01082719272A272B
:103EB0003B27C901B8011F910F910C947B1E0F93F2
:103EC0001F9300915A0310915B0320915C03309182
:103ED0005D03602B712B822B932B1F910F910C9400
:103EE0007B1E0F931F9300915A0310915B03209147
:103EF0005C0330915D0360237123822393231F9120
:103F00000F910C947B1E0F931F9300915A031091F5
:103F10005B0320915C0330915D036027712782274A
:103F200093271F910F910C947B1E08958F929F925F
:103F3000AF92BF92DF92EF92FF920F931F93CF93B6
:103F4000DF9300D000D01F92CDB7DEB76B837C83A8
:103F50008D838A018C819D81892B31F01F3F31F443
:103F600081E04F3F19F403C081E001C080E080FF91
:103F700003C080E090E04DC08B818823D1F1809018
:103F80005A0390905B03A0905C03B0905D03809116
:103F90005E0390915F03A0916003B0916103882A52
:103FA000992AAA2ABB2A8FE1E82EF12CD501C40157
:103FB0000E2C04C0B695A795979587950A94D2F7CD
:103FC00080FD06C081E0E81AF10880F7D12C07C017
:103FD000DE2CB8018E2D0E944106019799F388E0EE
:103FE000189FF0011124E652FD4FE00FF11DD08221
:103FF00009C088E0189FF0011124E652FD4FE00F40
:10400000F11DD08009831A8369817A818D2D0E94E8
:1040100041060F900F900F900F900F90DF91CF916E
:104020001F910F91FF90EF90DF90BF90AF909F9006
:104030008F90089590911501992379F1909116012F
:10404000992359F1982F9695969596959F31A1F0C1
:10405000E0911701F0911801E90FF11D877021E03F
:1040600030E0A90102C0440F551F8A95E2F7CA014A
:104070009181892B818308959091850390FF29C0B8
:104080001F928F9380E597E09F938F930E9438064D
:104090000F900F900F900F9008952091170130917D
:1040A0001801F90132969FEF40E05191851789F090
:1040B0009F3F19F4511101C0942F4F5F4E31A9F762
:1040C0009F3F39F0F901E90FF11D97FDFA958283C1
:1040D0000895089590911501992381F19091160109
:1040E000992361F1982F9695969596959F31A9F011
:1040F000E0911701F0911801E90FF11D877021E09F
:1041000030E0A90102C0440F551F8A95E2F7CA01A9
:10411000809591818923818308959091850390FFF3
:104120001CC01F928F9382E397E09F938F930E940E
:1041300038060F900F900F900F900895E09117019F
:10414000F09118019F01225E3F4F9281891301C0B7
:1041500012823196E217F307C1F7089581E090E0EB
:10416000E0911701F0911801E80FF91F10820196F4
:1041700080329105A9F70895809184030895909164
:104180008403892B80938403089580959091840300
:104190008923809384030895809384030895109263
:1041A0008403089590918303892B8093830308955A
:1041B00080959091830389238093830308951092BF
:1041C0008303089580936203089510926203089513
:1041D0008091170190911801FC0131969C01205E9D
:1041E0003F4F80E0919191118F5FE217F307D1F774
:1041F0000895E0911701F091180180918403808364
:10420000E0911701F0911801908180918303892B2F
:10421000808380916203882361F0E0911701F0911F
:1042200018019081892B80830E94E82081111092CF
:10423000620380911701909118010C94A11490933E
:1042400035018093340108958295982F937344E04B
:10425000949F900111248C7C86958695282B822F23
:104260008575880F2A7A2695822B08950895CF9315
:10427000DF9300D000D01F92CDB7DEB70F900F9024
:104280000F900F900F90DF91CF91089508950895AA
:104290000C94EB1580E0089583B7817F8C6083BF19
:1042A00083B7816083BF7894889583B78E7F83BFFF
:1042B0000895CF930E9422160E94270A0E94231677
:1042C000C0E08C2F0E940A0A811104C0CF5FC03168
:1042D000C1F701C081E0CF9108950E94100A0C94AB
:1042E0001D171F920F920FB60F9211248F939F9359
:1042F000AF93BF938091860390918703A091880329
:10430000B09189034196A11DB11D809386039093BE
:104310008703A0938803B0938903BF91AF919F91C6
:104320008F910F900FBE0F901F90189582E084BD63
:1043300093E095BD9AEF97BD80936E0008952FB7D7
:10434000F8948091860390918703A0918803B0919F
:1043500089032FBF08952FB7F89460918603709159
:10436000870380918803909189032FBF0895CF928E
:10437000DF92EF92FF920F931F932FB7F894409123
:1043800086035091870360918803709189032FBF42
:104390006A017B01EE24FF248C0120E030E0C0168E
:1043A000D106E206F30610F4415051099A01281B88
:1043B000390BC9011F910F91FF90EF90DF90CF90C3
:1043C00008951F920F920FB60F9211248F939F930F
:1043D000AF93BF938091860390918703A091880348
:1043E000B09189030196A11DB11D8093860390931E
:1043F0008703A0938803B0938903BF91AF919F91E6
:104400008F910F900FBE0F901F9018950E94D7119B
:10441000F89487E797E7909301088093000887E076
:1044200090EBDC018093980390939903A0939A03F7
:10443000B0939B039CE088E10FB6F894A895809315
:1044400060000FBE90936000FFCF80E090E0089581
:104450000895CF93C82F1F928F9384E797E09F937F
:104460008F930E94380681E090E0A0E0B0E0BC01AC
:10447000CD0104C0660F771F881F991FCA95D2F718
:104480000E94861E0F900F900F900F90CF910C946A
:104490001D17CF938732A8F58E3108F02BC18031DC
:1044A00009F49FC0F8F4873009F464C0A8F486309A
:1044B00009F024C180918503817F8E7F80938503DD
:1044C00089E797E00E949F058BE59AE00E949F058F
:1044D00081E080938A034CC08B30F1F18E3009F477
:1044E0006CC00CC1863109F4B0C020F4813109F4EC
:1044F000EDC004C1893109F491C08B3109F449C080
:10450000FDC0883349F150F4893209F4F1C0853394
:1045100009F4EEC0873209F0F1C0EAC0833409F42F
:10452000E7C028F48A3308F4E9C08953E4C088342A
:1045300009F0E4C00E941D178AE49AE00E949F05DA
:104540002FEF83ED90E3215080409040E1F700C0D1
:1045500000000E9406220CC084E997E05CC081E361
:104560009AE00E949F058091850381608093850376
:10457000C1E0C9C080918503C82FC17080FFEFCF13
:104580008DE39AE00E949F0580918503817F8E7F55
:104590003DC09091850391FBCC27C0F981E0C827ED
:1045A000892FC0FB81F980938503CC2319F084E225
:1045B0009AE027C086E19AE02EC09091850392FB95
:1045C000CC27C0F981E0C827892FC0FB82F98093EE
:1045D0008503CC2319F087E09AE013C087EF99E0B8
:1045E0001AC09091850393FBCC27C0F981E0C827BE
:1045F000892FC0FB83F980938503CC2351F08BEE88
:1046000099E00E949F0580918503816080938503D6
:104610007AC08EED99E00E949F05AACF8FEC99E0B9
:104620000E949F0589EA99E00E949F0581E699E032
:104630000E949F0589E399E00E949F058DEE98E016
:104640000E949F0582EC98E0E6CF84EB98E00E9400
:104650009F050E9495141F928F938AE998E09F937B
:104660008F930E943806809115011F928F9383E8E3
:1046700098E09F938F930E94380680918A021F9240
:104680008F9380E798E09F938F930E9438068091E4
:1046900016011F928F938DE598E09F938F930E9450
:1046A00038060E94AB219F938F937F936F9386E48C
:1046B00098E09F938F930E9438068DB79EB74696D9
:1046C0000FB6F8949EBF0FBE8DBF52CF0E941D172C
:1046D000C091160181E0C827C0931601CC2329F0B0
:1046E0008CE398E00E949F050EC081E398E093CF91
:1046F00080E001C08D510E9429223ACF8FE298E0DC
:104700000E949F05C0E08C2FCF91089580E008950E
:104710000C948623CF93C82F80918A03882319F0A5
:10472000813059F042C0E0911701F0911801808169
:10473000823261F08434D9F509C0E0911701F0911B
:1047400018018081823211F0843461F48C2F0E9430
:104750008823811104C08C2F0E94492224C081E04B
:1047600090E021C08C2F0E94862381111BC0C43190
:1047700089F018F4CB3029F010C0C93259F0C83391
:1047800061F489E797E00E949F0580E797E00E9427
:104790009F0508C010928A030CC08EE697E00E9425
:1047A0009F0507C081E0817006C010928A0380E0F7
:1047B00002C080E0F8CFCF910895EE0FFF1F059063
:0A47C000F491E02D0994F894FFCF66
:1047CA00013C0100000F69010000FFC00C2D0DC360
:1047DA000CF80CC40C01016303403622399A0664B2
:1047EA0006420609069505AE05C705E70500000855
:0447FA0000040002B5
:106800008800EA44E944E244040005000600070069
:10681000080009000A000B000C000D000E000F001C
:1068200010001100120013001400150016001700CC
:10683000180019001A001B001C001D001E001F007C
:10684000200021002200230024002500260027002C
:10685000280029002A002B002C002D002E002F00DC
:10686000300031003200330034003500360037008C
:10687000380039003A003B003C003D003E003F003C
:1068800040004100420043004400450046004700EC
:10689000480049004A004B004C004D004E004F009C
:1068A000500051005200530054005500560057004C
:1068B000580059005A005B005C005D005E005F00FC
:1068C00060006100620063006400F1A18500670060
:1068D000680069006A006B006C006D006E006F005C
:1068E0007000710072007300890087008A008B00BD
:1068F000E000E100E200E300E400E500E600E7007C
:106900000100010001000100EA4401000100E2442D
:106910000100010001000100460001004A004B0097
:10692000010001004700480001000100E9440100A6
:106930000100010001000100010001003A003B00DC
:106940003C003D003E003F0040004100420043004B
:10695000010035004C0039000100440045005200A0
:1069600049000100010050004F0029004D004E0079
:1069700051000100010001000100010001000100BF
:1069800001000100010001000100010001000100FF
:1069900001000100010001000100010001004D00A3
:1069A0004A004E004B0001000100010001000100FF
:1069B00001000100010001000100010001000100CF
:1069C00001000100010001000100010001000100BF
:1069D00001000100010001000100010001000100AF
:1069E0000100010001000100490001000100010057
:1069F000010001000100010001000100010001008F
:00000001FF
